:1000000009C016C015C03EC113C012C011C010C037
:100010000FC00EC011241FBECFE9CDBF20E0A0E667
:10002000B0E001C01D92AD36B207E1F795D1BDC178
:10003000E7CF806287B9369A3699FECF85B10895A9
:10004000E199FECF8EBB81E08CBB8DB30895E19921
:10005000FECF1CBA8EBB6DBB84E08CBBE19A0895C9
:100060008091620090E065E470E07AD18058934F0F
:1000700023E0959587952A95E1F728EB3BE0281B2F
:10008000390B3093610020936000C09A809160002A
:100090009091610041D1C098209160003091610041
:1000A00088E39AE4821B930B37C182E390E00FD17F
:1000B00081E087BB8AE088BB87E886B980E0C0DF43
:1000C0008093680082E0BCDF8093660080E096B396
:1000D0009A709230D9F482E0ACDF80936200909104
:1000E0006600891718F0915090936200B9DF81E0A3
:1000F000EECF82E09EDF80936200909168009817B7
:1001000018F09F5F90936200ABDF82E096B39A7025
:10011000983079F3813049F46091620080E097DF94
:1001200081E087DF682F81E009C0823041F460916F
:1001300062008DDF81E07DDF682F83E088DF80E073
:100140007FDF8093680081E07BDF8093670082E03F
:1001500077DF8093660083E073DF80936500909182
:100160006800809166009817C0F0109268001092A5
:1001700067008FEF809366008093650060E080E009
:1001800066DF6091670081E062DF6091660082E077
:100190005EDF6091650083E05ADF90916700809197
:1001A0006500981718F410926400089583E048DF02
:1001B0008093670081E044DF8093650081E0809355
:1001C0006400089586B38A708A3009F048C081E0DF
:1001D00030DFE82F8093630020916700F091650085
:1001E000821720F1F81768F130E090E0821B930B42
:1001F0006FEF70E0B5D06F2F70E0621B730BC1D052
:10020000862F90916400913009F4809520916800C8
:100210006091660070E0621B710990E0A1D06FEF01
:1002200070E0AFD0260F209362000BC08091640075
:10023000811103C08091680002C0809166008093A4
:100240006200FE1758F480916400811103C0809110
:10025000660002C0809168008093620001DF86B36F
:100260008A70823029F48091680080936200F8DE01
:1002700086B38A70883029F480916600809362008A
:10028000EFCE08951F920F920FB60F9211248F9305
:100290009F93AF93BF938091690090916A00A09162
:1002A0006B00B0916C000196A11DB11D8093690097
:1002B00090936A00A0936B00B0936C00BF91AF91D4
:1002C0009F918F910F900FBE0F901F9018950097E0
:1002D00041F0EFE5F9E03197F1F700C00000019738
:1002E000F6CF08959C0143E0369527954A95E1F7AE
:1002F000280F391F369527953695279588E0F8946D
:10030000C22FD32FE82FAC2FBD2F1197F1F700008C
:10031000E150C9F778940895009769F0883C9105F9
:100320000CF0E0CF03979C01220F331F96FD03C012
:10033000C9010197F1F7089583B7816083BF8FB535
:1003400083608FBD89B7826089BF12BE789417B869
:1003500086B1876886B90895EFDFA7DE33DFFECF69
:100360000024552704C0080E591F880F991F0097B5
:1003700029F076956795B8F37105B9F7802D952F1B
:100380000895AA1BBB1B51E107C0AA1FBB1FA617DC
:10039000B70710F0A61BB70B881F991F5A95A9F72E
:0E03A00080959095BC01CD010895F894FFCF93
:00000001FF
